:020000040000FA
:1000000085018316EC308500FF23900005308100C8
:100010009516151596168312073099008B1520300A
:100020008400DF008001840ADF08031D1228862077
:10003000B33081000B110A30BF006F20031D22284E
:10004000B50A1D2840210319272802212228480823
:100050003502031C022148083406031931286F2099
:100060002B285120491C9320FF303628AE0F4728FB
:10007000AE0A4C08AA002A0F05104D08AB002B0F42
:1000800085104E08AC002C0F05120B195621AA0A38
:1000900003190514AB0A03198514AC0A03190516D4
:1000A00036286B20B600013E0319662836308400DE
:1000B000840AB20A0319B30A6B2080003A3004069E
:1000C000031D5828B20A0319B30A08003008B20009
:1000D0003108B300512833088A00320882008F208B
:1000E000013E031978280530B0070318B10A6F28BC
:1000F000B40AB00A0319B10A8F20013E03198628F9
:100100003008B2003108B30003010800B401013027
:10011000B100B300CD30B000B200FF3808003108A4
:100120008A00300882003708C0003608BE00031D70
:10013000A1283808CC003908CD003A08CE00AD011E
:1001400008001330AD000130A000A100A2004C084F
:1001500038020318AE28A003A003003CA3004D08FA
:1001600039020318B628A103A103003CA4004E08DD
:100170003A020318BE28A203A203003CA5002308EC
:1001800024020318CA282308250225080318CF28AB
:100190002308CF28240825022508031C2408003C36
:1001A000A900A600A700A80008000130CA00092184
:1001B0002F088500851EDA280F30E92005080B106E
:1001C000630000005A30E920851ADA28851EE628E7
:1001D000002881010B110B1DEB28FF3E031DE928B0
:1001E000080083169A009B0A1C1555309D00AA3002
:1001F0009D009C148312080083169B0A1C141A0885
:1002000083120800CA0AC801B401C901CC01CD019A
:10021000CE010E21CA08031D092908004A08031946
:100220000800FF3E0319222983161C088312023995
:10023000031D08000008F120840A0408473A031946
:10024000CA0108003408C100C6004C08C200C60735
:100250004D08C300C6074E08C400C6074908C500BC
:100260004607003CC6004130840083169B01831280
:10027000CA0A08000408CB064B06CB068400080017
:1002800083169C1841299B01FC20C800C700FC2054
:10029000CC00C707FC20CD00C707FC20CE00C70755
:1002A000FC20C900C707FC20470708000108B33E2F
:1002B00081000B113A210E213A21C7080319662942
:1002C000BD0B6629C70B66290130CA00BC08031D97
:1002D000BC03851A6F29BB0A0319D5288D29FC3068
:1002E0003B0703187529BB018D29BC08031D802914
:1002F000BB010130C9066430BC000830C7008D293D
:100300006F205120CC01CD01CE0193200A30BF00D7
:10031000BB010830C700BC01C90149180800AD087D
:100320000319C129BE0B08003608BE0038084C0668
:10033000031D9C292D10A4292308A607031CA4290A
:100340002908A6072008CC0739084D06031DAA294D
:10035000AD10B2292408A707031CB2292908A70752
:100360002108CD073A084E06031DB8292D120800B2
:100370002508A807031C08002908A8072208CE079B
:100380000800C0080319CA29BF0B08000A30BF00C3
:10039000C00B080051209320080004340A34FF34B5
:1003A000FF34003404340A34013401340034FF349F
:1003B0000234073405340034003402340734003486
:1003C00000340034FF34053464340534053400341B
:1003D00001341934FF34FF340034013414340A3446
:1003E0000A3400340534C83402340234003405348D
:1003F000FF340034003400340234C8340234023490
:10040000003402346434003400340034023496344E
:100410000234023400346434FA34003400340034DA
:10042000FF340834C8344034403400340434643475
:10043000FF34FF3400340334143440344034003487
:1004400000340A34FF34FF34003400340334FF3402
:100450000134003400340534FF34FF3400340034F8
:100460000334FF340134003402340A3401340134DB
:1004700000340A34C8340134013400340A34C83436
:100480000134013400340A34C834013401340034F6
:100490000234FA344034403400340234FA34403404
:1004A000403400340234FA344034403400340234EE
:1004B000FA340134013400340234FA3401340134A2
:1004C00000340234FA340134013400340234FA3492
:1004D000FF34FF340034FF340034233440344034DC
:1004E000003400340134FF34FF340034003402346B
:1004F00005340534003400340134FF34FF34003453
:100500000034023405340534003400340134FF343F
:10051000FF34003400340234053405340034003430
:100520000134FF34FF340034003402340534053420
:1005300000340134C83440344034003403340034CF
:10054000C834C834003401340034FF34FF3400347C
:10055000013400349634963400340334003440348B
:10056000403400340134FA3440344034003402342E
:10057000B434203420340034013432344034403434
:100580000034FF34023407340034053400340234BC
:100590000734003400340034FF34003401340534AF
:1005A0000534003400341234003400340034003494
:1005B000013405340534003400340A340034003486
:1005C0000034003402340834083400340034073472
:1005D0000034003400340034023408340834003469
:1005E00000340234003400340034003464340C34F9
:1005F0000C3400341434C8340F340F340034013454
:10060000FA3419341934003401340A34643464344B
:100610000034053464341934193400340134FA34A4
:100620001934193400340134FA34193419340034CB
:10063000023432346034603400340834AF340F3460
:100640000F34003416347834033403340034003467
:10065000F034003400340034FF3400340134083402
:100660000834003400340C340034003400340034D6
:10067000023408340834003400340A3400340034BE
:1006800000340034053408340834003400340734AE
:1006900000340034003400340534083408340034A5
:1006A00000340334003400340034003464340C3437
:1006B0000C3400341434C834403440340034013431
:1006C00000342034FA34003401340034FA34203455
:1006D00000340134FA3440344034003401340034FE
:1006E000FA3420340034013400342034FA34003435
:1006F0000134FA3440344034003400340A34FA34DB
:10070000FA34003405340A344034403400340134BF
:10071000FA3440344034003416347834033403342B
:1007200000340034AF34003400340034FF34023479
:1007300007340534053400340234073400340034FF
:100740000034FF34FF34FF3FFF3FFF3FFF3FFF3FD9
:10075000FF3FFF3FFF3FFF3FFF3FFF3FFF3FFF3FA9
:10076000FF3FFF3FFF3FFF3FFF3FFF3FFF3FFF3F99
:10077000FF3FFF3FFF3FFF3FFF3FFF3FFF3FFF3F89
:10078000FF3FFF3FFF3FFF3FFF3FFF3FFF3FFF3F79
:10079000FF3FFF3FFF3FFF3FFF3FFF3FFF3FFF3F69
:1007A000FF3FFF3FFF3FFF3FFF3FFF3FFF3FFF3F59
:1007B000FF3FFF3FFF3FFF3FFF3FFF3FFF3FFF3F49
:1007C000FF3FFF3FFF3FFF3FFF3FFF3FFF3FFF3F39
:1007D000FF3FFF3FFF3FFF3FFF3FFF3FFF3FFF3F29
:1007E000FF3FFF3FFF3FFF3FFF3FFF3FFF3FFF3F19
:1007F000FF3FFF3FFF3FFF3FFF3FFF3FFF3F3834DB
:10420000FF00FF00FF00FF00FF00FF00FF00FF00B6
:10421000FF00FF00FF00FF00FF00FF00FF00FF00A6
:10422000FF00FF00FF00FF00FF00FF00FF00FF0096
:10423000FF00FF00FF00FF00FF00FF00FF00FF0086
:10424000FF00FF00FF00FF00FF00FF00FF00FF0076
:10425000FF00FF00FF00FF00FF00FF00FF00FF0066
:10426000FF00FF00FF00FF00FF00FF00FF00FF0056
:10427000FF00FF00FF00FF00FF00FF00FF00FF0046
:10428000FF00FF00FF00FF00FF00FF00FF00FF0036
:10429000FF00FF00FF00FF00FF00FF00FF00FF0026
:1042A000FF00FF00FF00FF00FF00FF00FF00FF0016
:1042B000FF00FF00FF00FF00FF00FF00FF00FF0006
:1042C000FF00FF00FF00FF00FF00FF00FF00FF00F6
:1042D000FF00FF00FF00FF00FF00FF00FF00FF00E6
:1042E000FF00FF00FF00FF00FF00FF00FF00FF00D6
:1042F000FF00FF00FF00FF00FF00FF00FF00FF00C6
:02400E00A40FFD
:08400000FF3FFF3FFF3FFF3FC0
:00000001FF
